:020000040000FA
:06000000FE300C303A282E
:08000800A000030E8301A1001A
:100010000A08A2008A01AA1503140B190310003064
:100020008100A30DA40DA50DA90B1F282A162508D4
:10003000A8002408A7002308A6001930A9008B10E7
:100040000B1122088A00210E8300A00E200E090049
:0C007400203084008001840A80300402E7
:10008000031C3C281F30CE000130CA00CB0080305A
:10009000CD000E30F4003230D70083161F308505B6
:1000A000003086050B3087058312850186018701A4
:1000B000103083168E008312703083168F008312E7
:1000C0000030031799000313003003179A0003133D
:1000D0000C30970000309F00003083169F00831281
:1000E000183003179E000313003003179F000313FB
:1000F000803083168100831211309000043092000A
:100100007F308316920083120030950000308316F2
:100110009400831223309400A63083169800831233
:10012000003083169B00831210309800193083161C
:1001300099008312003083168C00831200308316DE
:100140008D00831200308B000D16D62381018E01A5
:100150008F010B118B100B108C018D010D168B175D
:10016000E3211227311759219E22E920661AF02037
:10017000E61AEB202A1AF5208F080319B4288F01FC
:10018000E61A0717661A07155024B11B6821661A6C
:10019000F020E61AEB20AB239C2318227622661A65
:1001A000F020E61AEB204F18A221661AF020E61A7A
:1001B000EB204F18B428AA19E328CC0BB428AA1AAC
:1001C000E7281930A900AA110C30CC00B42851211D
:1001D000B428640008006B080E0203180713080017
:1001E0006B080E020318071108002A12C1302802FA
:1001F000031D05292708BE002608BD0007303E0262
:10020000031926278023D6234C29280827062602EF
:10021000031D0800F7302802031D11292708BF001D
:100220004C29A1302802031D18292708F0004C2969
:10023000A2302802031D1F292708C2004C29A7301D
:100240002802031D30292A10A71B2A1427087F39EA
:10025000EA002A1CEA012B142A1C2B10AB154C298E
:10026000C2302802031D4C292708C40064000D1E5B
:1002700037298B13440803178D0083168C130C1435
:1002800083120C080313C5008B177F3044022830FB
:100290000319C500CE164C29AA16AA110A30CC00A3
:1002A00008004F144F150B12831605118312051504
:1002B00008004F10CF101930A900AA12AA110A3055
:1002C000CC008316051583128B100B110B1608003A
:1002D000E71C080034080319080034083702031D1E
:1002E000772935083802031D7729B1130800AF0AB2
:1002F00001302F02031D7F293408930008000730C6
:100300002F02031D86293508930008000D302F02A7
:10031000031D9029360803190800360893000800C9
:100320000E302F02031D08003408B7003508B8004E
:10033000B401B501B601AF01B113311F08001C278C
:10034000311308004F19AF29C9030F304905031DA8
:100350000800C9080319AF290515C90E08000511C1
:100360004F11CF1859294B184608CB1847084B197D
:1003700048084D05031DBF294430C900C22911306A
:10038000C900C2290310CD0C0318C729080080300A
:10039000CD000310CB0DCB19CE2908000130CB00C6
:1003A0001030CE1ACA00410840028030031DCA0036
:1003B0000310CA0D03184A144A084E050319CE2922
:1003C000E321CF140800C601C701C8014A1CEE2969
:1003D0007730C6004008C700C100142ACA1CF5299E
:1003E0006630C6004308C700142A4A1DFC29553050
:1003F000C6007108C700142ACA1D032A4430C6006B
:100400007508C700142A4A1E0A2A3330C600770826
:10041000C700142ACA1E08002130C6004408C700BD
:100420004508C800CE12080046084706C800080064
:10043000051CB90A0518B903390803194012031934
:10044000B90A3C083902031940160319B903851C7F
:10045000BA0A8518BA033A080319C0110319BA0A6F
:100460003C083A020319C0150319BA03851DBB0ADB
:100470008519BB033B08031940110319BB0A3C084B
:100480003B02031940150319BB038719C010871DD0
:10049000C0143F1886163F1C8612C219BF23C2190A
:1004A000552A2A1BBF232A1F0712E7195C2ABF1CE3
:1004B0008613BF188617602ABF1C8617BF188613BD
:1004C0003F1F6613401C672A3F1B672AE617710807
:1004D000C01800306719F100C318752A2B1C752A43
:1004E000053077024310031C43140800B11B0800B9
:1004F000E008031D08003108420601390319872A64
:100500003013421830170C27311042183114301AAA
:10051000972A3108420602390319080030160C27C1
:10052000B110C218B114B2010530B3000800B20B0B
:100530000800B30B080030120C270800EA08031962
:10054000A82AAB18B02A6A0895002A18AA2A080017
:100550009501080006162B14AB10421AAB140800C4
:100560002B1D08002B11D518F72AD70BB4283230D1
:10057000D700D514AB19CF228B131D3003178D0074
:1005800083168C130C1483120C080313DE006A0804
:1005900095002A1C0800AB10421AAB140800AB11DE
:1005A0002130BF1C013E03178D0083168C130C14E1
:1005B00083120C080313D8008B17203003178D000B
:1005C00083168C130C1483120C080313DC008B1796
:1005D00058085C07D9005C07DA005C07DB006A0892
:1005E0007F3CDD000310DD0C0310DD0C0800DE088D
:1005F000031DFC2ADE03080058087702031C0E2B9B
:1006000059087702031C102B5A087702031C122B7F
:100610005B087702031C142BD40A162BD00A162B66
:10062000D10A162BD20A162BD30A162B50085104C6
:10063000520453045404103903190800D601501A07
:10064000D614511A5615521AD615531A5616541A4C
:10065000D616D001D101D201D301D401D510323048
:10066000D7006A08ED005D075619ED005D07D61941
:10067000ED005D07561AED005D07D61AED006D0816
:10068000950008000030BE007108BD0080230800FE
:10069000F10A720A71020318F1000800F103720AEC
:1006A000F11BF107080064000D1E542B8B1306305C
:1006B00003178D0083168C130C1483120C0803137C
:1006C0008B173F1D3030F200F203701B7D2B70083A
:1006D00071020318752B0319752B71087002BF186E
:1006E0007202BF18013EF300080070087102BF1CBF
:1006F0007202BF1C013EF3000800FA30F30008004C
:100700000D123E08831203178D00831203133D0858
:10071000831203178C00831603178C130C158B138D
:100720008B1B8F2B55308D00AA308D008C148B17AE
:100730000C11831203130800F40BA82B0E30F400E5
:100740009F147503F6009F18A32B2A151E08F500A9
:100750008D309F0008009F149F18AC2B2B158B1316
:1007600083161E0883128B17F7001E08C310031D83
:10077000C314FF30C318F70011309F000800AD13F9
:100780002D13AD0B0800AC0A03302C02031C08002B
:1007900007121E302E1C0A302C02031C0800AE0A61
:1007A0000130E71AAE000716AC01080064000D1E08
:1007B000D72B8B13003003178D0083168C130C146A
:1007C00083120C080313F1008B138B1BE42B0830EE
:1007D00003178D0083168C130C1483120C0803135B
:1007E000E7008B171C3003178D0083168C130C1435
:1007F00083120C080313BC008B1708000708403A4B
:10080000870008000708043A870008000708103A24
:10081000870008000608103A860008000608203AFB
:0C082000860008000608803A86000800E8
:1008A000123060020318E00104308A0060088207F9
:1008B0006A2C802C192D272D362D4F2D742D882D27
:1008C000B62DF02D2C2E572E6A2E782E872EA12E87
:1008D000B92EBE2E071707110612FA01FB01EB0114
:1008E000E6134010C0124013661B08003F1F0800AB
:1008F00066175323F308031908000130E0000800CD
:10090000AB104014B0170C272A17C31143138B13D5
:10091000053003178D0083168C130C1483120C08FA
:100920000313EC008B178B13033003178D00831612
:100930008C130C1483120C080313F8008B178B1301
:10094000043003178D0083168C130C1483120C08CB
:100950000313F9008B178B130C3003178D008316CC
:100960008C130C1483120C080313FC008B178B13CD
:100970000D3003178D0083168C130C1483120C0892
:100980000313FE008B178B130F3003178D00831694
:100990008C130C1483120C080313FD008B178B139C
:1009A0000E3003178D0083168C130C1483120C0861
:1009B0000313FF008B178B131B3003178D00831657
:1009C0008C130C1483120C080313E4008B178B1385
:1009D000133003178D0083168C130C1483120C082C
:1009E0000313E5008B170130BF1C013E8B13031767
:1009F0008D0083168C130C1483120C080313EF0064
:100A00008B171130BF1C013E8B1303178D0083160B
:100A10008C130C1483120C080313EE008B176C0854
:100A2000E100FF30EB000230E000EC080319202D5C
:100A30000800E616E10B08006C08E100EB0B08006B
:100A4000E6126508E100E2010330E0000800071348
:100A50000711E20B0800E10B08006C08E100EB0154
:100A60000430E000EC0803193E2D08006616E10B87
:100A700008006C08E100EB0F0800EB0366128B1313
:100A8000143003178D0083168C130C1483120C087A
:100A90000313E1008B17E2010530E00008000713A3
:100AA0000715E71C5F2DE10803195F2DE71F3016BE
:100AB000E71B30170C27E20B0800E10B0800E71FCB
:100AC0003012E71B30130C278B13163003178D00E1
:100AD00083168C130C1483120C080313E1008B177C
:100AE000E2010630E0000800E20B0800E10B08001C
:100AF0008B13183003178D0083168C130C1483127C
:100B00000C080313E1008B17E2010730E000080036
:100B1000C0160616AB156E08EA00AB14671CAB10C6
:100B2000E614F9262B14E20B0800E10B0800013053
:100B3000E61BF300AB1001307302031DA62D6E08F7
:100B4000EA00AB14671CAB10E610E6268B131930D5
:100B500003178D0083168C130C1483120C080313D7
:100B6000E1008B17E2010830E0000800C926780890
:100B700075020318C02D7F08FB02031CC52D080059
:100B80007F08FB070318DF2D0800FB010130E61B7F
:100B9000F300AB1001307302031DD52D6E08EA007F
:100BA000AB14671CAB10E610E626E20B0800E10B65
:100BB0000800C315F3012A131130E0000800FB01FF
:100BC0008B131A3003178D0083168C130C148312A9
:100BD0000C080313E1008B17E2010930E000080064
:100BE000C92679087502031CFA2D7F08FB02031C35
:100BF000FF2D08007F08FB070318092E0800FB01E2
:100C0000E20B0800E10B08004317F3011130E0008C
:100C10000800BF1C4823BF184E23F31B1C2EF30BE8
:100C20001C2E6E08EA00AB14671CAB10E610E6261B
:100C30000A30E000FA0108008B13193003178D0009
:100C400083168C130C1483120C080313E1008B170A
:100C5000E2010830E00008002A1D08002A1175088A
:100C60007602031C382E7C08FA02031C3F2E080073
:100C70007E08BF1C7D08FA070318412E0800FA0100
:100C80000800FA018712EA012B10AB10E0268B1343
:100C9000173003178D0083168C130C1483120C0865
:100CA0000313E1008B17E2010B30E0000800422340
:100CB000C0120612E20B0800B0130C27E10B08006B
:100CC000EC080319712E6C08E100FF30EB000C30CA
:100CD000E00008006616E10B08006C08E100EB0B71
:100CE000080066126508E100E2010D30E00008002E
:100CF00007130711E20B0800E10B08006C08E10084
:100D0000EB010E30E000EC0803198F2E0800E61608
:100D1000E10B08006C08E100EB0F0800EB03401743
:100D2000E6128B13153003178D0083168C130C14E9
:100D300083120C080313E1008B17E2010F30E0006F
:100D4000080007170711E71CB12EE1080319B12E9F
:100D5000671F3016671B30170C27E20B0800E10BEA
:100D60000800671F3012671B30130C271030E0009B
:100D700008002A13E0260030E00008002A13E026CD
:100D8000B0138712EA012B10AB1006120030E000FE
:100D90000800E61C0800E40B08008B131B30031747
:100DA0008D0083168C130C1483120C080313E400BB
:100DB0008B17EA0A6F086A02031D0800E610080094
:100DC0002430B4000030B500B11708002430B4005E
:100DD0008B131E3003178D0083168C130C14831293
:100DE0000C080313B6008B178A1512218A11B1174C
:100DF00008002430B4008B131F3003178D008316B6
:100E00008C130C1483120C080313B6008B178A156D
:100E100012218A11B11708000630B4003008B5005D
:100E2000B11708001430AF00FE30B400D930B5005F
:100E3000FF30B600B11708001430AF00FE30B40028
:100E4000E530B500FF30B600B1170800B701FE303D
:100E5000B400A130B5008A1500218A11B11708002D
:10120000B6013D18B617BD1836173D19B616BD19EB
:1012100036163D1AB615BD1A36153D1BB614BD1B44
:1012200036140800B5013618B517B6183517361933
:10123000B516B6193516361AB515B61A3515361B44
:06124000B514B601080020
:084000000B00000002000800A3
:02400E00CC03E1
:1042000000007E007E00AA0096000A001800FF0051
:104210008700FF00FF00FF0041002E0014002E0069
:1042200000003200320002001400150016003700B2
:104230000600190080005A00FF0000000100600025
:10424000050040004000FF00FF00FF00FF00FF00EE
:10425000FF00FF00FF00FF00FF00FF00FF00FF0066
:10426000FF00FF00FF00FF00FF00FF00FF00FF0056
:10427000FF00FF00FF00FF00FF00FF00FF00FF0046
:10428000FF00FF00FF00FF00FF00FF00FF00FF0036
:10429000FF00FF00FF00FF00FF00FF00FF00FF0026
:1042A000FF00FF00FF00FF00FF00FF00FF00FF0016
:1042B000FF00FF00FF00FF00FF00FF00FF00FF0006
:1042C000FF00FF00FF00FF00FF00FF00FF00FF00F6
:1042D000FF00FF00FF00FF00FF00FF00FF00FF00E6
:1042E000FF00FF00FF00FF00FF00FF00FF00FF00D6
:1042F000FF00FF00FF00FF00FF00FF00000028009C
:00000001FF
